BL51 BANKED LINKER/LOCATER V6.05                                                        07/29/2012  22:25:49  PAGE 1


BL51 BANKED LINKER/LOCATER V6.05, INVOKED BY:
D:\PROGRAM FILES\KEIL_51\C51\BIN\BL51.EXE Text1.obj TO xuanzhuan RAMSIZE (256)


MEMORY MODEL: SMALL


INPUT MODULES INCLUDED:
  Text1.obj (TEXT1)
  D:\PROGRAM FILES\KEIL_51\C51\LIB\C51S.LIB (?C_STARTUP)


LINK MAP OF MODULE:  xuanzhuan (TEXT1)


            TYPE    BASE      LENGTH    RELOCATION   SEGMENT NAME
            -----------------------------------------------------

            * * * * * * *   D A T A   M E M O R Y   * * * * * * *
            REG     0000H     0008H     ABSOLUTE     "REG BANK 0"
            DATA    0008H     0002H     UNIT         _DATA_GROUP_
            IDATA   000AH     0001H     UNIT         ?STACK

            * * * * * * *   C O D E   M E M O R Y   * * * * * * *
            CODE    0000H     0003H     ABSOLUTE     
            CODE    0003H     0570H     UNIT         ?CO?TEXT1
            CODE    0573H     0073H     UNIT         ?PR?MAIN?TEXT1
            CODE    05E6H     0012H     UNIT         ?PR?_DELAYUS?TEXT1
            CODE    05F8H     000CH     UNIT         ?C_C51STARTUP



OVERLAY MAP OF MODULE:   xuanzhuan (TEXT1)


SEGMENT                          DATA_GROUP 
  +--> CALLED SEGMENT          START    LENGTH
----------------------------------------------
?C_C51STARTUP                  -----    -----
  +--> ?PR?MAIN?TEXT1

?PR?MAIN?TEXT1                 0008H    0002H
  +--> ?CO?TEXT1
  +--> ?PR?_DELAYUS?TEXT1



SYMBOL TABLE OF MODULE:  xuanzhuan (TEXT1)

  VALUE           TYPE          NAME
  ----------------------------------

  -------         MODULE        TEXT1
  C:0000H         SYMBOL        _ICE_DUMMY_
  D:00A0H         PUBLIC        P2
  D:00B0H         PUBLIC        P3
  D:00C0H         PUBLIC        P4
  D:00C8H         PUBLIC        P5
BL51 BANKED LINKER/LOCATER V6.05                                                      07/29/2012  22:25:49  PAGE 2


  D:00A8H         PUBLIC        IE
  D:00B8H         PUBLIC        IP
  D:00D8H         PUBLIC        CCON
  C:0573H         PUBLIC        main
  D:0098H         PUBLIC        SCON
  D:0088H         PUBLIC        TCON
  C:05E6H         PUBLIC        _DelayUs
  C:0003H         PUBLIC        zimo
  B:00B0H.2       PUBLIC        KEY
  D:00D0H         PUBLIC        PSW
  -------         PROC          _DELAYUS
  D:0006H         SYMBOL        N
  -------         DO            
  D:0004H         SYMBOL        x
  -------         ENDDO         
  C:05E6H         LINE#         150
  C:05E6H         LINE#         151
  C:05E6H         LINE#         153
  C:05F7H         LINE#         154
  -------         ENDPROC       _DELAYUS
  -------         PROC          MAIN
  -------         DO            
  D:0002H         SYMBOL        i
  D:0008H         SYMBOL        j
  -------         ENDDO         
  C:0573H         LINE#         157
  C:0573H         LINE#         158
  C:0573H         LINE#         159
  C:057AH         LINE#         162
  C:057AH         LINE#         163
  C:057AH         LINE#         164
  C:057DH         LINE#         165
  C:057DH         LINE#         166
  C:0585H         LINE#         167
  C:058EH         LINE#         168
  C:058EH         LINE#         169
  C:0593H         LINE#         170
  C:0593H         LINE#         171
  C:05A7H         LINE#         172
  C:05A7H         LINE#         174
  C:05BCH         LINE#         175
  C:05CAH         LINE#         176
  C:05CFH         LINE#         177
  C:05D6H         LINE#         178
  C:05D9H         LINE#         179
  C:05DFH         LINE#         181
  -------         ENDPROC       MAIN
  -------         ENDMOD        TEXT1

Program Size: data=11.0 xdata=0 code=1540
LINK/LOCATE RUN COMPLETE.  0 WARNING(S),  0 ERROR(S)
